BL51 BANKED LINKER/LOCATER V5.03                                                        07/03/2006  12:26:16  PAGE 1


BL51 BANKED LINKER/LOCATER V5.03, INVOKED BY:
C:\KEIL\C51\BIN\BL51.EXE STARTUP.obj, SHTxx_Sample_Code.obj TO SHTxx_Demo2 RAMSIZE (256) CODE (0X0000-0X1FFF)


MEMORY MODEL: SMALL


INPUT MODULES INCLUDED:
  STARTUP.obj (?C_STARTUP)
  SHTxx_Sample_Code.obj (SHTXX_SAMPLE_CODE)
  C:\KEIL\C51\LIB\C51S.LIB (?C?CSTPTR)
  C:\KEIL\C51\LIB\C51S.LIB (?C?CSTOPTR)
  C:\KEIL\C51\LIB\C51S.LIB (?C?UIDIV)
  C:\KEIL\C51\LIB\C51S.LIB (?C?SIDIV)
  C:\KEIL\C51\LIB\C51S.LIB (?C?ILDPTR)
  C:\KEIL\C51\LIB\C51S.LIB (?C?ISTPTR)
  C:\KEIL\C51\LIB\C51S.LIB (?C?LMUL)
  C:\KEIL\C51\LIB\C51S.LIB (?C?SLCMP)
  C:\KEIL\C51\LIB\C51S.LIB (?C?ULSHR)
  C:\KEIL\C51\LIB\C51S.LIB (PRINTF)
  C:\KEIL\C51\LIB\C51S.LIB (?C?CLDPTR)
  C:\KEIL\C51\LIB\C51S.LIB (?C?CLDOPTR)
  C:\KEIL\C51\LIB\C51S.LIB (?C?PLDIIDATA)
  C:\KEIL\C51\LIB\C51S.LIB (?C?CCASE)
  C:\KEIL\C51\LIB\C51S.LIB (PUTCHAR)


LINK MAP OF MODULE:  SHTxx_Demo2 (?C_STARTUP)


            TYPE    BASE      LENGTH    RELOCATION   SEGMENT NAME
            -----------------------------------------------------

            * * * * * * *   D A T A   M E M O R Y   * * * * * * *
            REG     0000H     0008H     ABSOLUTE     "REG BANK 0"
                    0008H     0018H                  *** GAP ***
            BIT     0020H.0   0001H.1   UNIT         _BIT_GROUP_
                    0021H.1   0000H.7                *** GAP ***
            DATA    0022H     001CH     UNIT         _DATA_GROUP_
            IDATA   003EH     0001H     UNIT         ?STACK

            * * * * * * *   C O D E   M E M O R Y   * * * * * * *
            CODE    0000H     0003H     ABSOLUTE     
                    0003H     07FDH                  *** GAP ***
            CODE    0800H     035CH     UNIT         ?PR?PRINTF?PRINTF
            CODE    0B5CH     01FDH     UNIT         ?C?LIB_CODE
            CODE    0D59H     00CAH     UNIT         ?PR?MAIN?SHTXX_SAMPLE_CODE
            CODE    0E23H     00BFH     UNIT         ?PR?_CALC_SHT10?SHTXX_SAMPLE_CODE
            CODE    0EE2H     0088H     UNIT         ?PR?_S_MEASURE?SHTXX_SAMPLE_CODE
            CODE    0F6AH     002EH     UNIT         ?PR?_S_READ_BYTE?SHTXX_SAMPLE_CODE
            CODE    0F98H     002DH     UNIT         ?PR?_S_WRITE_BYTE?SHTXX_SAMPLE_CODE
            CODE    0FC5H     0027H     UNIT         ?PR?PUTCHAR?PUTCHAR
            CODE    0FECH     001EH     UNIT         ?CO?SHTXX_SAMPLE_CODE
            CODE    100AH     0019H     UNIT         ?PR?S_TRANSSTART?SHTXX_SAMPLE_CODE
            CODE    1023H     0011H     UNIT         ?PR?S_CONNECTIONRESET?SHTXX_SAMPLE_CODE
            CODE    1034H     000DH     UNIT         ?PR?INIT_UART?SHTXX_SAMPLE_CODE
            CODE    1041H     000CH     UNIT         ?C_C51STARTUP

BL51 BANKED LINKER/LOCATER V5.03                                                      07/03/2006  12:26:16  PAGE 2




OVERLAY MAP OF MODULE:   SHTxx_Demo2 (?C_STARTUP)


SEGMENT                                            BIT_GROUP          DATA_GROUP 
  +--> CALLED SEGMENT                           START    LENGTH     START    LENGTH
-----------------------------------------------------------------------------------
?C_C51STARTUP                                   -----    -----      -----    -----
  +--> ?PR?MAIN?SHTXX_SAMPLE_CODE

?PR?MAIN?SHTXX_SAMPLE_CODE                      -----    -----      0022H    0008H
  +--> ?PR?INIT_UART?SHTXX_SAMPLE_CODE
  +--> ?PR?S_CONNECTIONRESET?SHTXX_SAMPLE_CODE
  +--> ?PR?_S_MEASURE?SHTXX_SAMPLE_CODE
  +--> ?PR?_CALC_SHT10?SHTXX_SAMPLE_CODE
  +--> ?CO?SHTXX_SAMPLE_CODE
  +--> ?PR?PRINTF?PRINTF

?PR?S_CONNECTIONRESET?SHTXX_SAMPLE_CODE         -----    -----      -----    -----
  +--> ?PR?S_TRANSSTART?SHTXX_SAMPLE_CODE

?PR?_S_MEASURE?SHTXX_SAMPLE_CODE                -----    -----      002AH    0009H
  +--> ?PR?S_TRANSSTART?SHTXX_SAMPLE_CODE
  +--> ?PR?_S_WRITE_BYTE?SHTXX_SAMPLE_CODE
  +--> ?PR?_S_READ_BYTE?SHTXX_SAMPLE_CODE

?PR?_CALC_SHT10?SHTXX_SAMPLE_CODE               -----    -----      002AH    000CH

?PR?PRINTF?PRINTF                               0020H.0  0001H.1    002AH    0014H
  +--> ?PR?PUTCHAR?PUTCHAR



SYMBOL TABLE OF MODULE:  SHTxx_Demo2 (?C_STARTUP)

  VALUE           TYPE          NAME
  ----------------------------------

  -------         MODULE        ?C_STARTUP
  C:1041H         SEGMENT       ?C_C51STARTUP
  I:003EH         SEGMENT       ?STACK
  C:0000H         PUBLIC        ?C_STARTUP
  D:00E0H         SYMBOL        ACC
  D:00F0H         SYMBOL        B
  D:0083H         SYMBOL        DPH
  D:0082H         SYMBOL        DPL
  N:0000H         SYMBOL        IBPSTACK
  N:0100H         SYMBOL        IBPSTACKTOP
  N:0080H         SYMBOL        IDATALEN
  C:1044H         SYMBOL        IDATALOOP
  N:0000H         SYMBOL        PBPSTACK
  N:0000H         SYMBOL        PBPSTACKTOP
  N:0000H         SYMBOL        PDATALEN
  N:0000H         SYMBOL        PDATASTART
  N:0000H         SYMBOL        PPAGE
  N:0000H         SYMBOL        PPAGEENABLE
BL51 BANKED LINKER/LOCATER V5.03                                                      07/03/2006  12:26:16  PAGE 3


  D:00A0H         SYMBOL        PPAGE_SFR
  D:0081H         SYMBOL        SP
  C:1041H         SYMBOL        STARTUP1
  N:0000H         SYMBOL        XBPSTACK
  N:0000H         SYMBOL        XBPSTACKTOP
  N:0000H         SYMBOL        XDATALEN
  N:0000H         SYMBOL        XDATASTART
  C:0000H         LINE#         92
  C:1041H         LINE#         99
  C:1043H         LINE#         100
  C:1044H         LINE#         101
  C:1045H         LINE#         102
  C:1047H         LINE#         151
  C:104AH         LINE#         155
  -------         ENDMOD        ?C_STARTUP

  -------         MODULE        SHTXX_SAMPLE_CODE
  C:0000H         SYMBOL        _ICE_DUMMY_
  D:00B0H         PUBLIC        P3
  C:0E23H         PUBLIC        _calc_sht10
  B:00B0H.5       PUBLIC        DATA
  C:0D59H         PUBLIC        main
  C:0EE2H         PUBLIC        _s_measure
  C:100AH         PUBLIC        s_transstart
  C:1023H         PUBLIC        s_connectionreset
  D:0098H         PUBLIC        SCON
  D:0089H         PUBLIC        TMOD
  D:0088H         PUBLIC        TCON
  D:008DH         PUBLIC        TH1
  C:1034H         PUBLIC        init_uart
  B:00B0H.4       PUBLIC        SCK
  C:0F6AH         PUBLIC        _s_read_byte
  C:0F98H         PUBLIC        _s_write_byte
  -------         PROC          _S_WRITE_BYTE
  D:0007H         SYMBOL        value
  -------         DO            
  D:0005H         SYMBOL        i
  D:0006H         SYMBOL        error
  -------         ENDDO         
  C:0F98H         LINE#         37
  C:0F98H         LINE#         40
  C:0F98H         LINE#         41
  C:0F9AH         LINE#         42
  C:0FA2H         LINE#         43
  C:0FAAH         LINE#         44
  C:0FACH         LINE#         45
  C:0FAEH         LINE#         46
  C:0FB1H         LINE#         47
  C:0FB3H         LINE#         48
  C:0FB9H         LINE#         49
  C:0FBBH         LINE#         50
  C:0FBDH         LINE#         51
  C:0FC1H         LINE#         52
  C:0FC3H         LINE#         53
  C:0FC4H         LINE#         54
  -------         ENDPROC       _S_WRITE_BYTE
  -------         PROC          _S_READ_BYTE
BL51 BANKED LINKER/LOCATER V5.03                                                      07/03/2006  12:26:16  PAGE 4


  D:0007H         SYMBOL        ack
  -------         DO            
  D:0005H         SYMBOL        i
  D:0006H         SYMBOL        val
  -------         ENDDO         
  C:0F6AH         LINE#         57
  C:0F6AH         LINE#         60
  C:0F6AH         LINE#         61
  C:0F6CH         LINE#         62
  C:0F6EH         LINE#         63
  C:0F76H         LINE#         64
  C:0F78H         LINE#         65
  C:0F7EH         LINE#         66
  C:0F80H         LINE#         67
  C:0F86H         LINE#         68
  C:0F8CH         LINE#         69
  C:0F8EH         LINE#         70
  C:0F91H         LINE#         71
  C:0F93H         LINE#         72
  C:0F95H         LINE#         73
  C:0F97H         LINE#         74
  -------         ENDPROC       _S_READ_BYTE
  -------         PROC          S_TRANSSTART
  C:100AH         LINE#         77
  C:100AH         LINE#         84
  C:100AH         LINE#         85
  C:100EH         LINE#         86
  C:100FH         LINE#         87
  C:1011H         LINE#         88
  C:1012H         LINE#         89
  C:1014H         LINE#         90
  C:1015H         LINE#         91
  C:1017H         LINE#         92
  C:101AH         LINE#         93
  C:101CH         LINE#         94
  C:101DH         LINE#         95
  C:101FH         LINE#         96
  C:1020H         LINE#         97
  C:1022H         LINE#         98
  -------         ENDPROC       S_TRANSSTART
  -------         PROC          S_CONNECTIONRESET
  -------         DO            
  D:0007H         SYMBOL        i
  -------         ENDDO         
  C:1023H         LINE#         101
  C:1023H         LINE#         108
  C:1023H         LINE#         110
  C:1027H         LINE#         111
  C:1029H         LINE#         112
  C:102BH         LINE#         113
  C:102DH         LINE#         114
  C:1031H         LINE#         115
  -------         ENDPROC       S_CONNECTIONRESET
  -------         PROC          _S_MEASURE
  D:002AH         SYMBOL        p_value
  D:002DH         SYMBOL        p_checksum
  D:0030H         SYMBOL        mode
BL51 BANKED LINKER/LOCATER V5.03                                                      07/03/2006  12:26:16  PAGE 5


  -------         DO            
  D:0031H         SYMBOL        error
  D:0082H         SYMBOL        i
  -------         ENDDO         
  C:0EE2H         LINE#         120
  C:0EE8H         LINE#         123
  C:0EE8H         LINE#         124
  C:0EEDH         LINE#         127
  C:0EF0H         LINE#         128
  C:0EF8H         LINE#         129
  C:0EFCH         LINE#         130
  C:0F10H         LINE#         131
  C:0F10H         LINE#         132
  C:0F10H         LINE#         133
  C:0F2CH         LINE#         134
  C:0F37H         LINE#         135
  C:0F46H         LINE#         136
  C:0F58H         LINE#         137
  C:0F67H         LINE#         138
  C:0F69H         LINE#         139
  -------         ENDPROC       _S_MEASURE
  -------         PROC          INIT_UART
  C:1034H         LINE#         142
  C:1034H         LINE#         145
  C:1037H         LINE#         146
  C:103AH         LINE#         147
  C:103DH         LINE#         148
  C:1040H         LINE#         149
  -------         ENDPROC       INIT_UART
  -------         PROC          _CALC_SHT10
  D:002AH         SYMBOL        p_humidity
  D:002DH         SYMBOL        p_temperature
  -------         DO            
  D:0030H         SYMBOL        rh
  D:0006H         SYMBOL        t
  D:0032H         SYMBOL        t_C
  D:0034H         SYMBOL        rh_lin
  -------         ENDDO         
  C:0E23H         LINE#         153
  C:0E29H         LINE#         160
  C:0E29H         LINE#         161
  C:0E31H         LINE#         162
  C:0E3CH         LINE#         168
  C:0E45H         LINE#         173
  C:0E50H         LINE#         174
  C:0E50H         LINE#         175
  C:0E69H         LINE#         176
  C:0E87H         LINE#         177
  C:0E89H         LINE#         179
  C:0E89H         LINE#         181
  C:0EB5H         LINE#         182
  C:0EC6H         LINE#         183
  C:0EC6H         LINE#         187
  C:0ED4H         LINE#         188
  -------         ENDPROC       _CALC_SHT10
  -------         PROC          MAIN
  -------         DO            
BL51 BANKED LINKER/LOCATER V5.03                                                      07/03/2006  12:26:16  PAGE 6


  D:0022H         SYMBOL        humi_val
  D:0024H         SYMBOL        temp_val
  D:0026H         SYMBOL        error
  D:0027H         SYMBOL        checksum
  D:0028H         SYMBOL        i
  -------         ENDDO         
  C:0D59H         LINE#         192
  C:0D59H         LINE#         200
  C:0D59H         LINE#         205
  C:0D5CH         LINE#         207
  C:0D5FH         LINE#         208
  C:0D5FH         LINE#         209
  C:0D5FH         LINE#         210
  C:0D62H         LINE#         211
  C:0D7AH         LINE#         212
  C:0D93H         LINE#         213
  C:0D9AH         LINE#         215
  C:0D9AH         LINE#         216
  C:0DACH         LINE#         217
  C:0DFEH         LINE#         218
  C:0DFEH         LINE#         221
  -------         ENDPROC       MAIN
  -------         ENDMOD        SHTXX_SAMPLE_CODE

  -------         MODULE        ?C?CSTPTR
  C:0B5CH         PUBLIC        ?C?CSTPTR
  -------         ENDMOD        ?C?CSTPTR

  -------         MODULE        ?C?CSTOPTR
  C:0B6EH         PUBLIC        ?C?CSTOPTR
  -------         ENDMOD        ?C?CSTOPTR

  -------         MODULE        ?C?UIDIV
  C:0B90H         PUBLIC        ?C?UIDIV
  -------         ENDMOD        ?C?UIDIV

  -------         MODULE        ?C?SIDIV
  C:0BE5H         PUBLIC        ?C?SIDIV
  -------         ENDMOD        ?C?SIDIV

  -------         MODULE        ?C?ILDPTR
  C:0C1BH         PUBLIC        ?C?ILDPTR
  -------         ENDMOD        ?C?ILDPTR

  -------         MODULE        ?C?ISTPTR
  C:0C46H         PUBLIC        ?C?ISTPTR
  -------         ENDMOD        ?C?ISTPTR

  -------         MODULE        ?C?LMUL
  C:0C65H         PUBLIC        ?C?LMUL
  -------         ENDMOD        ?C?LMUL

  -------         MODULE        ?C?SLCMP
  C:0CB4H         PUBLIC        ?C?SLCMP
  -------         ENDMOD        ?C?SLCMP

  -------         MODULE        ?C?ULSHR
BL51 BANKED LINKER/LOCATER V5.03                                                      07/03/2006  12:26:16  PAGE 7


  C:0CCAH         PUBLIC        ?C?ULSHR
  -------         ENDMOD        ?C?ULSHR

  -------         MODULE        PRINTF
  D:002AH         PUBLIC        ?_PRINTF517?BYTE
  D:002AH         PUBLIC        ?_PRINTF?BYTE
  D:002AH         PUBLIC        ?_SPRINTF517?BYTE
  D:002AH         PUBLIC        ?_SPRINTF?BYTE
  C:0862H         PUBLIC        _PRINTF
  C:0862H         PUBLIC        _PRINTF517
  C:085CH         PUBLIC        _SPRINTF
  C:085CH         PUBLIC        _SPRINTF517
  -------         ENDMOD        PRINTF

  -------         MODULE        ?C?CLDPTR
  C:0CDDH         PUBLIC        ?C?CLDPTR
  -------         ENDMOD        ?C?CLDPTR

  -------         MODULE        ?C?CLDOPTR
  C:0CF6H         PUBLIC        ?C?CLDOPTR
  -------         ENDMOD        ?C?CLDOPTR

  -------         MODULE        ?C?PLDIIDATA
  C:0D23H         PUBLIC        ?C?PLDIIDATA
  -------         ENDMOD        ?C?PLDIIDATA

  -------         MODULE        ?C?CCASE
  C:0D33H         PUBLIC        ?C?CCASE
  -------         ENDMOD        ?C?CCASE

  -------         MODULE        PUTCHAR
  C:0FC5H         PUBLIC        _PUTCHAR
  -------         ENDMOD        PUTCHAR

******************************************************************************
* RESTRICTED VERSION WITH 0800H BYTE CODE SIZE LIMIT; USED: 02E0H BYTE (35%) *
******************************************************************************

Program Size: data=38.1 xdata=0 code=2128
LINK/LOCATE RUN COMPLETE.  0 WARNING(S),  0 ERROR(S)
